:100000000C94280018950000189500001895000021
:10001000189500001895000018950000189500002C
:10002000189500000C94220C1895000018950000FB
:10003000189500001895000018950000189500000C
:1000400018950000189500001895000018950000FC
:100050008FE181BD87E181BD8FE58DBFC4E0E8E719
:100060004E2E88E08EBFD8E0F7E05F2EEEEFF7E08F
:10007000A0E6B0E088278D933197E9F783E389B94B
:1000800088E18AB9662487E08ABB87EF8BBB8FEB58
:1000900087BB8FEB88BB80EE84BB8FEF85BB80E88E
:1000A00081BB8BE382BB80E08FBD81E08EBD8FE1A1
:1000B00081BD87E181BD86E086B980E487B9C398B8
:1000C000C29AD89AC498C798C598F894A895709180
:1000D0006B00706270936B000027ABE6B0E08C9110
:1000E00085FB0EF401E041E0041711F00C947C0054
:1000F00087E88ABB87E78BBB0E94680D7091D000B0
:1001000078607093D000EFEFF1E0A1ECB0E091E007
:100110000E9447280091C100003081E009F080E092
:100120008F930091C1000E3F80E010F009F081E054
:100130009F91892B882311F40C94A1008EEB80935E
:10014000C1000091C1004AE0040F01BF82E390E0CA
:100150000E940A27E0EFF0E50E945126ABE6B0E0EE
:100160008C9185FBA8E6B7E00E942F278D93882706
:100170008C930E9449260E945D26EAE0F0E0BB27AE
:10018000A0E10E9444280D3311F40C94FD00EBE033
:10019000F0E0A0E1BB2788E08C937BE70E94332846
:1001A000ECE0F0E001E010E0A0E1BB277BE70E947B
:1001B0003528EAE0F0E0A0E1BB278DE38C937BE7F4
:1001C0000E943328EEE0F0E0A0E1BB2780E08C93B2
:1001D0007BE70E943328E0E1F0E000E010E0A0E1DE
:1001E000BB277BE70E943528EFE0F0E0A0E1BB27CA
:1001F00080E08C937BE70E943328EBE0F0E0ACEBEF
:10020000B0E00E9444280091BC000C3318F011F0BB
:100210000C940C010C940F018CE38093BC0080E7DC
:1002200097E9ADEBB0E08D939C93ECE0F0E0A7EBA9
:10023000B0E00E944628EEE0F0E0A2ECB0E00E94C0
:100240004428EFE0F0E0A3ECB0E00E9444280E94D4
:100250006C0DE0E1F0E0A4E6B0E00E944628A4E6E0
:10026000B0E00E94CC25E0E1F0E0A4E6B0E07BE75E
:100270000E943528A7EBB0E00D911C91003050E0B2
:10028000150711F00C944A0181E090E0A7EBB0E073
:100290008D939C93E8E0F1E50E945126A8E6B7E033
:1002A000ECEBF0E00E949D270E944926E0E1F1E599
:1002B0000E945126A8E6B7E0E7EBF0E00E948E2707
:1002C0000E944926E0E1F1E50E945126A8E6B7E048
:1002D000E2ECF0E00E949D270E944926E0E1F1E572
:1002E0000E945126A8E6B7E0E3ECF0E00E949D27CB
:1002F0000E944926E0E1F1E50E945126A8E6B7E018
:10030000E4E6F0E00E948E270E944926E0E1F1E554
:100310000E945126BB27A3E38C9180FBA8E6B7E09F
:100320000E942F278D9388278C930E9449260E9434
:100330005D260027BB27A3E38C9180FB0EF401E030
:1003400041E0041711F00C94B10170916B007B7FB8
:1003500070936B00A2ECB0E08C918E7F8C930C9428
:10036000BB0170916B00746070936B00A2ECB0E005
:100370008C9181608C930027BB27A3E38C9183FB36
:100380000EF401E041E0041711F00C94D3017091D8
:10039000D0007F7D7093D000A2ECB0E08C918D7F77
:1003A0008C930C94DD017091D00070627093D0003A
:1003B000A2ECB0E08C9182608C9381E882BB80E0FB
:1003C0008093600081E08093620000916200083CAD
:1003D00018F011F00C940C020027BB27A0E38C91BD
:1003E00080FB0EF401E040E0041718F011F00C94CB
:1003F000FB010C940002A0E6B0E08C918F5F8C931F
:1004000081E090E00E940A27A2E6B0E08C918F5F25
:100410008C9311F00C94E50100916000003011F014
:100420000C944802E2E1F1E50E9451260E945D260B
:1004300070916B007F7D70936B0070916B007064A6
:1004400070936B0081E08093620000916200043041
:1004500018F011F00C944602979A84E690E00E94FE
:100460000A27979889E190E00E940A2787E38ABBD0
:1004700087EC8BBB80E384BB8FEC85BBA2E6B0E04E
:100480008C918F5F8C9311F00C9425020C94560282
:10049000ECE1F1E50E9451260E945D2670916B000F
:1004A0007F7B70936B0080E882BB979880E080939D
:1004B000CF0070916B007D7F70936B0080E0809324
:1004C000C50086E08093BF008DE08093C00084E18A
:1004D00090E00E940A270E94F626C49AE6E2F1E51F
:1004E0000E9451260E945D2688EC90E00E940A2717
:1004F000A89581B5886181BD877F81BDE0E6F0E088
:10050000FA93EA930E94491B2296A89500916000F5
:10051000003011F40C9498020E948B1AE0E3F1E58C
:100520000E9451260E945D260E94320D0C949D026D
:100530007091D0007F7E7093D000EAE3F1E50E94D5
:1005400051260E94B41A84E690E00E940A270027F0
:10055000A0EDB0E08C9184FB0EF401E040E00417C4
:1005600011F00C94B5020E944C108FEF0E9460268F
:1005700082E390E00E940A277894A89581B588606C
:1005800081BDA3EBB0E04D915C91A7EBB0E00D9184
:100590001C910417150718F011F00C94D1020C945B
:1005A000D70281E090E0A7EBB0E08D939C93002709
:1005B000ABE6B0E08C9182FB0EF401E041E0041761
:1005C00081E009F080E08F930027A0EDB0E08C91EE
:1005D00084FB0EF401E040E0041781E009F080E0C4
:1005E0009F918923882311F40C940903E7EBF0E031
:1005F000FA93EA935A924A9280E0A42DB52D8C93F7
:1006000081E00E94B9250E94210E249681E00E947B
:10061000B52580E08093B90080E080936A000027D0
:10062000A0EDB0E08C9184FB0EF401E041E00417F2
:1006300011F00C941D030E94680DA8950E9441269C
:10064000ACE6B0E08D9388278C930091CF0000300A
:1006500081E009F080E08F930027BB27A3E38C9112
:1006600081FB0EF401E041E0041781E009F080E035
:100670009F91892B882311F40C945A030027ABE631
:10068000B0E08C9186FB0EF401E041E0041711F01C
:100690000C945303E3E6F0E0FA93EA930E945A19AC
:1006A00022960C945A03E3E6F0E0FA93EA930E9450
:1006B0000F19229681E090E00E940A270091CF0056
:1006C000003081E009F080E08F930027ABE6B0E0D6
:1006D0008C9181FB0EF401E041E0041781E009F008
:1006E00080E09F91892B882311F40C947B0385E093
:1006F00090E00E940A27ACE6B0E08C91803081E067
:1007000009F480E08F9300916300003081E009F4E8
:1007100080E09F91892B8F930091B900013081E097
:1007200009F080E09F91892B882311F40C940F032A
:1007300000916300003011F40C94D5050E94160D51
:100740000027BB27A3E38C9182FB0EF401E041E07C
:10075000041711F00C943C048EB5887F8EBD8AE09E
:1007600090E00E940A270027ABE6B0E08C9186FB60
:100770000EF401E041E0041711F00C94D003E3E61D
:10078000F0E0FA93EA930E945A192296A3E6B0E0A9
:100790008C91A7EBB0E08D9388278C930C9409047F
:1007A000E3E6F0E0FA93EA930E940F192296009193
:1007B0006300003011F40C940904A3E6B0E08C91BE
:1007C000A7EBB0E08D9388278C93009163000430F1
:1007D00011F00C94F10383E090E0A7EBB0E08D936F
:1007E0009C9300916300083011F00C94FD0384E0A9
:1007F00090E0A7EBB0E08D939C93009163000031F3
:1008000011F00C94090485E090E0A7EBB0E08D9323
:100810009C93A3EBB0E04D915C91A7EBB0E00D9100
:100820001C910417150780E010F009F081E08F9308
:10083000A7EBB0E00D911C91003050E0150781E06E
:1008400009F080E09F91892B882311F40C942E04E9
:1008500081E090E0A7EBB0E08D939C930091630062
:10086000003011F40C943A04ACE6B0E0E4E4F1E5B5
:100870000E9430260C94D5050027ABE6B0E08C91A1
:1008800086FB0EF401E041E0041711F00C944105E1
:10089000E3E6F0E0FA93EA930E945A192296009157
:1008A00063000D3011F00C945B04ACE6B0E0E6E4BC
:1008B000F1E50E943026009163000F3011F00C9496
:1008C000A304ABEDB0E00E94E727A4E6B0E00D93EF
:1008D0001C93A3EBB0E04D915C91A4E6B0E00D91C8
:1008E0001C910417150718F011F00C9479040C945E
:1008F0007F0481E090E0A4E6B0E08D939C93A4E6B1
:10090000B0E00D911C91003050E0150711F00C94EF
:100910009104ACE6B0E0E8E4F1E50E9430260C94E6
:100920009F04A4E6B0E08D919C91A7EBB0E08D937D
:100930009C93ACE6B0E0E4E4F1E50E943026ABED38
:10094000B0E088278C9300916300013011F00C9483
:10095000B104ABEDB0E00E943626EAE4F1E50E9476
:10096000302600916300023011F00C94BF04ABED0F
:10097000B0E00E943626ECE4F1E50E9430260091BA
:100980006300033011F00C94CD04ABEDB0E00E9495
:100990003626EEE4F1E50E94302600916300053032
:1009A00011F00C94DB04ABEDB0E00E943626E0E5DC
:1009B000F1E50E94302600916300063011F00C949E
:1009C000E904ABEDB0E00E943626E2E5F1E50E94D5
:1009D000302600916300073011F00C94F704ABED62
:1009E000B0E00E943626E4E5F1E50E943026009151
:1009F0006300093011F00C940505ABEDB0E00E94E6
:100A00003626E6E5F1E50E943026009163000A30C3
:100A100011F00C941305ABEDB0E00E943626E8E52A
:100A2000F1E50E943026009163000B3011F00C9428
:100A30002105ABEDB0E00E943626EAE5F1E50E9423
:100A40003026009163000E3011F00C942F05ABEDB1
:100A5000B0E00E943626ECE5F1E50E943026ABEDD1
:100A6000B0E00E945E28082F033018F011F00C94BB
:100A70003B050C943F05ABEDB0E088278C930C94BC
:100A80006C05E3E6F0E0FA93EA930E940F192296D0
:100A900000916300013011F00C945405ACE6B0E015
:100AA000E8E4F1E50E94302600916300023011F085
:100AB0000C946005ACE6B0E0EEE5F1E50E9430266E
:100AC00000916300043011F00C946C05ACE6B0E0CA
:100AD000E6E4F1E50E94302600916300083011F051
:100AE0000C94A2050091BC00033018F011F00C9496
:100AF0007B050C94A205ACEBB0E08C9183508C93F9
:100B00008EB5887F8EBD5A924A928091BC00A42DEA
:100B1000B52D8C9381E00E94B9250E943722229640
:100B200081E00E94B525EBE0F0E0ACEBB0E07BE7C4
:100B30000E9433280091CF00013011F00C94A205DF
:100B400081E08EBD00916300003111F00C94D50559
:100B50000091BC00063410F00C94D505ACEBB0E06D
:100B60008C918D5F8C938EB5887F8EBD5A924A9200
:100B70008091BC00A42DB52D8C9381E00E94B925F5
:100B80000E943722229681E00E94B525EBE0F0E03A
:100B9000ACEBB0E07BE70E9433280091CF0001303E
:100BA00011F00C94D50581E08EBDECE6F0E0ACE6EA
:100BB000B0E00E9423270091B900013011F00C949D
:100BC000020680E08093B900ACE6B0E0E8E4F1E52D
:100BD0000E9430260027A0EDB0E08C9185FB0EF43A
:100BE00001E041E0041711F00C94020681E090E06E
:100BF000A7EBB0E08D939C93ACE6B0E0E4E4F1E5C4
:100C00000E943026ACE6B0E0E0E6F1E50E94642800
:100C100011F00C9449065A924A928091BF00A42D7B
:100C2000B52D8C9381E00E94B9255A924A92809109
:100C3000C000A42DB52D8C9381E00E94B9250E949F
:100C40009022249682E00E94B5250091C30041E0E5
:100C5000042BA0E6B0E00C937091D0007460709308
:100C6000D0008EB5887F8EBDEFE0F0E0A0E6B0E06A
:100C70007BE70E943328809160008093C30000913D
:100C8000CF00013011F00C94470681E08EBD0C942A
:100C9000CC0BE2E6F1E50E94642811F00C948C067E
:100CA0005A924A9280E0A42DB52D8C9381E00E9447
:100CB000B9255A924A9280E0A42DB52D8C9381E0FB
:100CC0000E94B9250E949022249682E00E94B525B8
:100CD0000091C3004EEF0423A0E6B0E00C937091A6
:100CE000D0007B7F7093D0008EB5887F8EBDEFE003
:100CF000F0E0A0E6B0E07BE70E943328809160003E
:100D00008093C3000091CF00013011F00C948A064B
:100D100081E08EBD0C94CC0BE4E4F1E50E946428E4
:100D200011F00C94F7060091CF00013011F00C94F3
:100D30009B060E94160DA3EBB0E04D915C91A7EBD2
:100D4000B0E00D911C910417150718F011F00C94E8
:100D5000F5060027A0EDB0E08C9184FB0EF401E0D5
:100D600040E0041711F00C94C806E7EBF0E0FA93AA
:100D7000EA935A924A9280E0A42DB52D8C9381E09B
:100D80000E94B9250E94210E249681E00E94B5257B
:100D90000027A0EDB0E08C9184FB0EF401E041E06F
:100DA000041711F00C94F5060E94320D0027A0EDF7
:100DB000B0E08C9184FB0EF401E040E0041711F0E8
:100DC0000C94F506E7EBF0E0FA93EA935A924A9214
:100DD00080E0A42DB52D8C9381E00E94B9250E945E
:100DE000210E249681E00E94B5250C94CC0BE4E6FC
:100DF000F1E50E94642811F00C9405070E94160D7D
:100E000080E08093C5000C94CC0BE6E4F1E50E94F1
:100E1000642811F00C943F070091CF00013011F0CD
:100E20000C943D070027ABE6B0E08C9181FB0EF4FB
:100E300001E040E0041711F00C942F078EB5887F75
:100E40008EBD89B78B7F89BF70916B007260709384
:100E50006B0084E690E00E940A270C943D07709195
:100E60006B007D7F70936B0080E29EE49DBD8CBD26
:100E700081E08EBD89B7846089BF0C94CC0BE8E417
:100E8000F1E50E94642811F00C94D7070091CF007F
:100E9000013011F00C944E070E94160DA7EBB0E044
:100EA0000E94CC250027A0EDB0E08C9183FB0EF4CE
:100EB00001E041E0041711F00C9473070027ABE642
:100EC000B0E08C9182FB0EF401E040E0041711F0D9
:100ED0000C946E07A7EBB0E00E94D2257091D00071
:100EE000777F7093D000A3EBB0E04D915C91A7EBBE
:100EF000B0E00D911C910417150718F011F00C9437
:100F000083070C94890781E090E0A7EBB0E08D9314
:100F10009C930027A0EDB0E08C9184FB0EF401E0DF
:100F200040E0041711F00C94A807E7EBF0E0FA9307
:100F3000EA935A924A9280E0A42DB52D8C9381E0D9
:100F40000E94B9250E94210E249681E00E94B525B9
:100F50000027A0EDB0E08C9184FB0EF401E041E0AD
:100F6000041711F00C94D5070E94320D0027A0ED54
:100F7000B0E08C9184FB0EF401E040E0041711F026
:100F80000C94D507E7EBF0E0FA93EA935A924A9271
:100F900080E0A42DB52D8C9381E00E94B9250E949C
:100FA000210E249681E00E94B5250C94CC0BEEE531
:100FB000F1E50E94642811F00C944F080091CF00D5
:100FC000013011F00C94E6070E94160DA7EBB0E07B
:100FD0000D911C91013050E0150718F011F00C94A0
:100FE000F3070C94F907A7EBB0E00E94D2250C940C
:100FF0000108A3EBB0E08D919C91A7EBB0E08D933D
:101000009C930027A0EDB0E08C9184FB0EF401E0EE
:1010100040E0041711F00C942008E7EBF0E0FA939D
:10102000EA935A924A9280E0A42DB52D8C9381E0E8
:101030000E94B9250E94210E249681E00E94B525C8
:101040000027A0EDB0E08C9184FB0EF401E041E0BC
:10105000041711F00C944D080E94320D0027A0EDEA
:10106000B0E08C9184FB0EF401E040E0041711F035
:101070000C944D08E7EBF0E0FA93EA935A924A9207
:1010800080E0A42DB52D8C9381E00E94B9250E94AB
:10109000210E249681E00E94B5250C94CC0BE6E647
:1010A000F1E50E94642811F00C94C208A7EBB0E0AF
:1010B0000E94CC25A3EBB0E04D915C91A7EBB0E092
:1010C0000D911C910417150718F011F00C946A0883
:1010D0000C94700881E090E0A7EBB0E08D939C93B6
:1010E0008EB5887F8EBDA3E7B0E00D911D912D9147
:1010F0003C91A3E9B0E00D931D932D933C93002701
:10110000A0EDB0E08C9184FB0EF401E040E0041708
:1011100011F00C94B8085A924A92A3E9B0E00D91EC
:101120001D912D913C91A42DB52D0D931D932D93C3
:101130003C9384E00E94B9255A924A92A7EBB0E012
:101140008D919C91A42DB52D8D939C9382E00E944E
:10115000B9255A924A9280E0A42DB52D8C9381E056
:101160000E94B9250E945B11269687E00E94B52552
:101170000091CF00013011F00C94C00881E08EBDC9
:101180000C94CC0BE8E6F1E50E94642811F00C9475
:101190003609A7EBB0E00D911C91013050E0150726
:1011A00018F011F00C94D6080C94DC08A7EBB0E012
:1011B0000E94D2250C94E408A3EBB0E08D919C91A1
:1011C000A7EBB0E08D939C938EB5887F8EBDA3E78F
:1011D000B0E00D911D912D913C91A3E9B0E00D93EC
:1011E0001D932D933C930027A0EDB0E08C9184FBE0
:1011F0000EF401E040E0041711F00C942C095A920F
:101200004A92A3E9B0E00D911D912D913C91A42D3E
:10121000B52D0D931D932D933C9384E00E94B92529
:101220005A924A92A7EBB0E08D919C91A42DB52DD6
:101230008D939C9382E00E94B9255A924A9280E055
:10124000A42DB52D8C9381E00E94B9250E945B11DD
:10125000269687E00E94B5250091CF00013011F05D
:101260000C94340981E08EBD0C94CC0BEAE6F1E5D8
:101270000E94642811F00C944609ECE0F0E0A7EB22
:10128000B0E07BE70E9435280C94CC0BECE6F1E54E
:101290000E94642811F00C945A098DE181BD85E10A
:1012A00081BD0E94160D81B5886081BD0C945609E0
:1012B0000C94CC0BACE6B0E0EEE6F1E50E946428BD
:1012C00081E008F480E08F93ACE6B0E0E0E7F1E580
:1012D0000E94642881E010F009F080E09F9189234A
:1012E000882311F40C942E0A89B78B7F89BF8EB5A1
:1012F000887F8EBD0E943D26A0E6B0E08C930091D1
:101300006000003011F40C947A090E944126A7EB8A
:10131000B0E08D9388278C9380E08093CF0070910C
:101320006B007D7F70936B00A3EBB0E04D915C91FF
:10133000A7EBB0E00D911C910417150780E010F0A9
:1013400009F081E08F93A7EBB0E00D911C91003084
:1013500050E0150781E009F080E09F91892B8823F8
:1013600011F40C94CE0981E090E0A7EBB0E08D93EE
:101370009C93E7EBF0E0FA93EA935A924A9281E069
:10138000A42DB52D8C9381E00E94B9250E94210ED9
:10139000249681E00E94B5250C942C0A0027A0ED2C
:1013A000B0E08C9184FB0EF401E040E0041781E092
:1013B00009F080E08F93ACE6B0E0EEE6F1E50E9444
:1013C000642881E009F080E09F918923882311F44B
:1013D0000C94FD09E7EBF0E0FA93EA935A924A92F3
:1013E00081E0A42DB52D8C9381E00E94B9250E9447
:1013F000210E249681E00E94B5250027A0EDB0E0E3
:101400008C9184FB0EF401E040E0041781E009F0C8
:1014100080E08F93ACE6B0E0E0E7F1E50E9464285D
:1014200081E009F080E09F918923882311F40C94D6
:101430002C0AE7EBF0E0FA93EA935A924A9280E0A2
:10144000A42DB52D8C9381E00E94B9250E94210E18
:10145000249681E00E94B5250C94CC0BE2E7F1E5DF
:101460000E94642811F00C94690A0E943D26A0E6AF
:10147000B0E08C9300916000003011F40C94350AB8
:101480000E944126ACEBB0E08C938EB5887F8EBD78
:101490005A924A928091BC00A42DB52D8C9381E084
:1014A0000E94B9250E943722229681E00E94B5252C
:1014B000EBE0F0E0ACEBB0E07BE70E94332800917A
:1014C000CF00013011F00C94670A81E08EBD0C94BE
:1014D000CC0BE4E7F1E50E94642811F00C94B70A04
:1014E0000E943D26A0E6B0E08C93009160000030A1
:1014F00011F40C94700A8091C200809360000E94E5
:101500004126A2ECB0E08C93A2ECB0E08C918F73FA
:101510008C930E946C0D0091C20040E10423A0E670
:10152000B0E00C9300916000003111F00C949C0A23
:101530000E94680D0C949E0A0E946A0DA2ECB0E015
:101540008C918F7E8C938EB5887F8EBDEEE0F0E01F
:10155000A2ECB0E07BE70E9433280091CF0001307D
:1015600011F00C94B50A81E08EBD0C94CC0BE6E72B
:10157000F1E50E94642811F00C941B0B0091C2004D
:101580004FE30423A0E6B0E00C930091CF000130BC
:1015900011F00C94D00AA0E6B0E08C9180588C93A6
:1015A0000027A0EDB0E08C9184FB0EF401E041E057
:1015B000041711F00C94E10AA0E6B0E08C91805C75
:1015C0008C930027ABE6B0E08C9181FB0EF401E038
:1015D00041E0041711F00C94F20AA0E6B0E08C91FF
:1015E000805E8C938091B700809362008EB5887F77
:1015F0008EBD31E0A0E6B0E00E94582631E0ACEBB1
:10160000B0E00E94582631E0A2E6B0E00E945826E1
:101610008091B3008093620031E0A2E6B0E00E94C6
:1016200058260091CF00013011F00C94190B81E085
:101630008EBD0C94CC0BE8E7F1E50E94642811F014
:101640000C949E0BA6EDB0E00D911D912D913C9157
:10165000A2EDB0E04D915D916D917C910E94762755
:10166000A6E6B0E00D931D932D933D93A6E6B0E062
:101670000E94BD25A6E6B0E00D911D912D913C91F3
:1016800040E052E060E070E00E946A26A6E6B0E02A
:101690000D931D932D933D93A6E6B0E00D911D9102
:1016A0002D913C91A4ECB0E04C915527662777270B
:1016B0000E946F26A6E6B0E04D935D936D937D93F7
:1016C000A6E6B0E00D911D912D913C914AE050E0CD
:1016D00060E070E00E946F26A6E6B0E04D935D9357
:1016E0006D937D9344E150E060E070E0A6E6B0E0E9
:1016F0000D911D912D913C910E947B270CF402C00D
:101700000C948C0B00E010E020E030E0A6E6B0E0A6
:101710000D931D932D933C938EB5887F8EBD34E041
:10172000A6E6B0E00E9458260091CF00013011F0EB
:101730000C949C0B81E08EBD0C94CC0BEAE7F1E598
:101740000E94642811F00C94B60B8EB5887F8EBD74
:10175000A5EAB0E00E944B260091CF00013011F0C5
:101760000C94B40B81E08EBD0C94CC0BECE7F1E54E
:101770000E94642811F00C94CC0B8EB5887F8EBD2E
:101780000E94F7100091CF00013011F00C94CA0BA9
:1017900081E08EBD0C94CC0B81E090E00E940A2782
:1017A00000916300003011F40C94200CA8950027E0
:1017B000ABE6B0E08C9186FB0EF401E041E004174B
:1017C00011F00C94EC0BE3E6F0E0FA93EA930E943C
:1017D0005A1922960C94F30BE3E6F0E0FA93EA939D
:1017E0000E940F19229681E090E00E940A27009142
:1017F0006300003011F00C94D60B0091CF00013043
:1018000081E009F080E08F930027ABE6B0E08C9197
:1018100081FB0EF401E041E0041781E009F080E073
:101820009F91892B882311F40C941C0C83E090E089
:101830000E940A270C94200C8AE090E00E940A275C
:101840000C940F030F921F922F923F924F925F9230
:101850007F928F929F92AF92BF920F931F932F937D
:101860003F934F935F936F937F938F939F93AF9328
:10187000BF93CF93DF93EF93FF938FB78F93F8943A
:1018800089B78B7F89BF8EB5887F8EBD5A924A9269
:1018900080E092E0A42DB52D8D939C9382E00E9470
:1018A000B9250E943325229682E00E94B525009139
:1018B000DA000A3011F00C945F0C0E94680D0E944F
:1018C0007D1E0091DA000A3011F00C946C0C0E941D
:1018D0006A0D80E08093DA00AAEDB0E08C918F5F12
:1018E0008C93A8950027A0EDB0E08C9184FB0EF4BA
:1018F00001E040E0041711F00C94910C5A924A92C6
:1019000080E092E0A42DB52D8D939C9382E00E94FF
:10191000B9250E943325229682E00E94B5250E94B7
:101920007D1EA6EDB0E04D915D916D917C91A2ED93
:10193000B0E00D911D912D913C910E947B2780E09C
:101940000CF481E08F930027A0EDB0E08C9184FB34
:101950000EF401E040E0041781E009F080E09F917F
:101960008923882311F40C94C00C80E49CE99DBD6C
:101970008CBD81E08EBD89B7846089BF0C94F60C64
:1019800080E08093CF0070916B007D7F70936B003F
:101990000027A0EDB0E08C9184FB0EF401E040E064
:1019A000041711F00C94DD0CABE6B0E08C9182FBD7
:1019B000A9EBB0E0882780F98C930091C2004FE733
:1019C0000423A1E6B0E00C930E946A0D80E08093AE
:1019D000C5000027ABE6B0E08C9185FB0EF401E07A
:1019E00041E0041711F00C94F60CDF988F918FBF33
:1019F000FF91EF91DF91CF91BF91AF919F918F9127
:101A00007F916F915F914F913F912F911F910F9116
:101A1000BF90AF909F908F907F905F904F903F903E
:101A20002F901F900F901895F894FFCF89B78B7F58
:101A300089BF8EB5887F8EBD80E08093CF00709186
:101A40006B007D7F70936B000027ABE6B0E08C915C
:101A500085FB0EF401E041E0041711F00C94310D08
:101A6000DF9808956E98C498C598C7980E946A0D2B
:101A7000E2E0F0E00E946426C49A0E94F62684E622
:101A800090E00E940A27A8957091D0007F7E709305
:101A9000D000E0E6F0E0FA93EA930E94491B229618
:101AA00000916000003011F40C94650D7091D0002D
:101AB00070617093D00084E690E00E940A276E98CF
:101AC000C498C598C7980C94670D0E944C1008954F
:101AD00097980895979A089581E00E941927709128
:101AE0006B007B7F70936B000091C20041E0042388
:101AF000A881B9810C93A881B9810C91003011F4AF
:101B00000C94870D70916B00746070936B007091F2
:101B1000D0007F7D7093D0000091C20042E004238A
:101B2000A881B9810C93A881B9810C91003011F47E
:101B30000C949F0D7091D00070627093D0007091E2
:101B4000D0007F7B7093D0000091C20044E004235A
:101B5000A881B9810C93A881B9810C91003011F44E
:101B60000C94B70D7091D00070647093D000709198
:101B7000D0007F777093D0000091C20048E004232A
:101B8000A881B9810C93A881B9810C91003011F41E
:101B90000C94CF0D7091D00070687093D00070914C
:101BA0006B00777F70936B000091C20040E20423CA
:101BB000A881B9810C93A881B9810C91003011F4EE
:101BC0000C94E70D70916B00786070936B007091CE
:101BD000D0007B7F7093D0000091C30041E00423CC
:101BE000A881B9810C93A881B9810C91003011F4BE
:101BF0000C94FF0D7091D00074607093D000009130
:101C0000C30046E00423A881B9810C93A881B9815F
:101C10000C9142E00E944E280C93A881B9818C91CE
:101C20008093D1000091D100033011F00C941B0E71
:101C300082E08093D10081E0481A8827580A2296D2
:101C4000089582E00E94192781E00E9419278EB52D
:101C5000887F8EBD70916B007D7F70936B00A3E7D2
:101C6000B0E00D911D912D913C91A3E9B0E00D9351
:101C70001D932D933C935A924A92A3E9B0E00D91A3
:101C80001D912D913C91A42DB52D0D931D932D9358
:101C90003C9384E00E94B9255A924A92AA85BB855A
:101CA0008D919C91A42DB52D8D939C9382E00E94E3
:101CB000B9255A924A9280E0A42DB52D8C9381E0EB
:101CC0000E94B9250E945B11269687E00E94B525E7
:101CD00040E050E060E070E0AFE8B0E00D911D91B1
:101CE0002D913C910E947B2711F00C94790E0C945D
:101CF00046100E94EB215A924A928091BC00A42D7A
:101D0000B52D8C9381E00E94B9250E94372222963E
:101D100081E00E94B5255A924A92ADEBB0E08D91D8
:101D20009C91A42DB52D8D939C9382E00E94B925A2
:101D30000E94CF22229682E00E94B5250027A0EDC6
:101D4000B0E08C9182FB0EF401E041E0041711F049
:101D50000C94C40E5A924A928091BF00A42DB52DC6
:101D60008C9381E00E94B9255A924A928091C000DA
:101D7000A42DB52D8C9381E00E94B9250E9490225C
:101D8000249682E00E94B525A3E9B0E00D911D9153
:101D90002D913C91A2EDB0E00D931D932D933C93BA
:101DA000A3E9B0E00D911D912D913C91AFE8B0E019
:101DB0004D915D916D917C910E947127A6EDB0E0EF
:101DC0000D931D932D933D9380E0A881B9818C9351
:101DD0000E947D1E81E090E0AA81BB818D939C933F
:101DE000AA81BB810D911C910F3F51E0150718F09E
:101DF00011F00C942A0FAA81BB81AD90BC90AFED7D
:101E0000B0E0AA0DBB1D0C910F3F81E009F080E00E
:101E10008F93AA81BB81AD90BC90A0EEB0E0AA0DDB
:101E2000BB1D0C910F3E80E010F009F081E09F9106
:101E30008923882311F40C94230F81E0A881B981B0
:101E40008C930C942A0FAA81BB810E94CC2511F09F
:101E50000C94F00EA881B9810C91013011F00C9412
:101E6000E80EAA81BB81AD90BC90A1EEB0E0AA0DB6
:101E7000BB1D8C91AA81BB818D9388278C93AA81ED
:101E8000BB810D911C9140E150E00E94EA25AA819E
:101E9000BB814D935C9380E18093C400AA81BB8198
:101EA0000D911C91013050E0150711F00C945D0F5D
:101EB00084E08093C4000C94EA0F023050E01507D0
:101EC00011F00C94680F85E08093C4000C94EA0F25
:101ED000033050E0150711F00C94730F86E08093E7
:101EE000C4000C94EA0F043050E0150711F00C9474
:101EF0007E0F87E08093C4000C94EA0F053050E019
:101F0000150711F00C94890F88E08093C4000C949D
:101F1000EA0F063050E0150711F00C94940F8AE098
:101F20008093C4000C94EA0F073050E0150711F0BD
:101F30000C949F0F8CE08093C4000C94EA0F08303F
:101F400050E0150711F00C94AA0F8EE08093C400A6
:101F50000C94EA0F093050E0150711F00C94B50FFE
:101F600080E18093C4000C94EA0F0A3050E015071A
:101F700011F00C94C00F84E18093C4000C94EA0F1C
:101F80000B3050E0150711F00C94CB0F88E18093D3
:101F9000C4000C94EA0F0C3050E0150711F00C94BB
:101FA000D60F8CE18093C4000C94EA0F0D3050E002
:101FB000150711F00C94E10F80E28093C4000C949B
:101FC000EA0F0E3050E0150711F00C94EA0F88E28A
:101FD0008093C400AFE8B0E00D911D912D913C912C
:101FE00040E052E060E070E00E946A26A6E6B0E0C1
:101FF0000D931D932D933D93A6E6B0E00D911D9199
:102000002D913C91A4ECB0E04C91552766277727A1
:102010000E946F26A6E6B0E04D935D936D937D938D
:10202000A6E6B0E00D911D912D913C9148EE53E054
:1020300060E070E00E946F26A6E6B0E04D935D93ED
:102040006D937D93AC81BD810C91003011F00C94A7
:1020500046100027ABE6B0E08C9185FB0EF401E062
:1020600041E0041711F00C943610DF9A81E0809360
:10207000CF0088EC9FEA9DBD8CBD89B7846089BF85
:1020800081E08EBD85E090E00E940A2783E0481A37
:102090008827580A24960895A895A3E7B0E00D91E3
:1020A0001D912D913C91A7E7B0E00D931D932D93C9
:1020B0003C93A3E7B0E00D911D912D913C91A3E9D4
:1020C000B0E00D931D932D933C935A924A92A3E94D
:1020D000B0E00D911D912D913C91A42DB52D0D9346
:1020E0001D932D933C9384E00E94B9255A924A9205
:1020F00080E090E0A42DB52D8D939C9382E00E940A
:10210000B9255A924A9280E0A42DB52D8C9381E096
:102110000E94B9250E945B11269687E00E94B52592
:10212000A895A3EBB0E00D911C91013050E015078C
:1021300010F00C94C2105A924A9281E0A42DB52D51
:102140008C9381E00E94B9250E942923229681E088
:102150000E94B5258CE291E00E940A275A924A9289
:1021600080E0A42DB52D8C9381E00E94B9250E94BA
:102170002923229681E00E94B5257091D0007061DC
:102180007093D000A895A3E7B0E00D911D912D911B
:102190003C91A3E9B0E00D931D932D933C93A7EBE5
:1021A000B0E00D911C91003050E0150781E009F07E
:1021B00080E08F93A3EBB0E04D915C91A7EBB0E092
:1021C0000D911C910417150780E010F009F081E0D3
:1021D0009F91892B882311F40C94F41081E090E0F6
:1021E000A7EBB0E08D939C930E946A0D089584E064
:1021F0000E941927A2EDB0E00D911D912D913C9107
:10220000A881B9810D931D932D933C93A3E7B0E072
:102210000D911D912D913C91A3E9B0E00D931D937B
:102220002D933C935A924A92A3E9B0E00D911D91EF
:102230002D913C91A42DB52D0D931D932D933C9381
:1022400084E00E94B9255A924A928FE19EE4A42D1F
:10225000B52D8D939C9382E00E94B9255A924A92A3
:1022600080E0A42DB52D8C9381E00E94B9250E94B9
:102270005B11269687E00E94B525A3E7B0E00D919B
:102280001D912D913C91A3E9B0E00D931D932D93E9
:102290003C93A881B9810D911D912D913C91A2EDA6
:1022A000B0E00D931D932D933C9384E0481A88274A
:1022B000580A2296089581E00E94192781E00E9421
:1022C000192781E00E94192780E090E0A5EBB0E09B
:1022D0008D939C9370916B007F7E70936B0000E0F8
:1022E00010E020E030E0AFE8B0E00D931D932D93B7
:1022F0003C930027ABE6B0E08C9183FB0EF401E049
:1023000041E0041781E009F080E08F93A885B9854A
:102310000D911C91003050E0150781E009F480E038
:102320009F9189238F93AE81BF810C91003081E012
:1023300009F080E09F918923882311F40C94FB110C
:10234000A7E9B0E0E885F9850E948E27E7E9F0E08B
:10235000A8E6B7E00E941928E8E6F7E0A7E9B0E0B0
:102360001127222704E033270E94332781E4AC8120
:10237000BD818C93AC81BD818C9180939D0081E067
:10238000E7E9F0E001E00A93ACE6B0E00E941E2825
:10239000ACE6B0E08C91AEE9B0E08C9382E0E7E986
:1023A000F0E001E00A93ACE6B0E00E941E28ACE643
:1023B000B0E08C91AFE9B0E08C9383E0E7E9F0E026
:1023C00001E00A93ACE6B0E00E941E28ACE6B0E063
:1023D0008C91A0EAB0E08C9384E0E7E9F0E001E0C2
:1023E0000A93ACE6B0E00E941E28ACE6B0E08C9107
:1023F000A1EAB0E08C9389B78B7F89BF8EB5887FC7
:102400008EBD81B5886181BD877F81BDABECB0E0B9
:102410000D911D912D913C91A7ECB0E00D931D9372
:102420002D933C93A7E7B0E04D915D916D917C9128
:10243000A3E7B0E00D911D912D913C910E947B2767
:1024400011F00C942D1202E010E020E030E0A7EC37
:10245000B0E00D931D932D933C9380E0A881B9814A
:102460008C93EA81FB81FA93EA935A924A92AE8561
:10247000BF850D911D912D913C91A42DB52D0D93EE
:102480001D932D933C9384E00E94B9250E947420F3
:10249000249684E00E94B525AA81BB810C910E3F51
:1024A00011F40C945F127091D00070617093D000A1
:1024B00070916B00706170936B000C9472125A9261
:1024C0004A92AA85BB858D919C91A42DB52D8D93A3
:1024D0009C9382E00E94B9250E947313229682E0A9
:1024E0000E94B525A881B9818C918F5F8C93409112
:1024F0007000A881B9810C91041781E009F080E097
:102500008F930027ABE6B0E08C9184FB0EF401E0E2
:1025100041E0041781E009F480E09F91892388233A
:1025200011F40C94281300917F000B3011F00C94DF
:10253000D512E7ECF0E0FA93EA935A924A92A7ECAC
:10254000B0E00D911D912D913C91A42DB52D0D93D1
:102550001D932D933C9384E00E94B9250E94B317EC
:10256000249684E00E94B525EA85FB85FA93EA93D8
:102570005A924A92A7ECB0E00D911D912D913C9199
:10258000A42DB52D0D931D932D933C9384E00E94B3
:10259000B9250E944917249684E00E94B52580E061
:1025A000A881B9818C930C942613A7E7B0E04D91D4
:1025B0005D916D917C91A3E7B0E00D911D912D91FE
:1025C0003C910E947B2711F00C94EC12AA85BB85EC
:1025D0000E94BD250C942613E7ECF0E0FA93EA93F1
:1025E0005A924A92A7ECB0E00D911D912D913C9129
:1025F000A42DB52D0D931D932D933C9384E00E9443
:10260000B9250E94B317249684E00E94B525EA8577
:10261000FB85FA93EA935A924A92A7ECB0E00D91A7
:102620001D912D913C91A42DB52D0D931D932D93AE
:102630003C9384E00E94B9250E944917249684E0C7
:102640000E94B52580E0A881B9818C930C942C134D
:10265000AA85BB850E94BD250027ABE6B0E08C9122
:1026600084FB0EF401E041E0041711F00C943112E8
:10267000C49AA885B9850D911C91003050E01507CA
:1026800011F00C944B13A5EBB0E08D919C91A3EB52
:10269000B0E08D939C930091CF00013081E009F070
:1026A00080E08F930027A0EDB0E08C9184FB0EF4C6
:1026B00001E040E0041781E009F080E09F91892368
:1026C000882311F40C946D1380E593EC9DBD8CBDB3
:1026D00081E08EBD89B7846089BF83E0481A88276E
:1026E000580A2696089584E00E94192784E00E94E3
:1026F000192781E00E94192781E00E94192781E0B3
:102700000E94192781E00E94192780E0AE81BF81D5
:102710008C93AE81BF810C910F3018F011F00C94A6
:10272000561581E0AC81BD818C93AC81BD810C914B
:102730000C3018F011F00C94B5138FEF0E94FD26A9
:102740000E94FF260E94FE26AC81BD81AD90BB2475
:10275000A1E8B0E0AA0DBB1D8C93AC81BD818C912A
:102760008F5F8C9311F00C9495138DE0AC81BD813B
:102770008C93AC81BD810C91043118F011F00C9454
:10278000D3138FEF0E94FD260E94FF260E94FE2693
:10279000A881B9818C93AC81BD818C918F5F8C9322
:1027A00011F00C94B913EA85FB85FA93EA93EA8554
:1027B000FB85FA93EA930E94DE1524960027ABE688
:1027C000B0E08C9184FB0EF401E041E0041711F0BD
:1027D0000C94EC130C944E1580E0AA81BB818C9371
:1027E00000918D00003281E009F080E08F9300912C
:1027F0008D00003181E009F080E09F91892B8823D2
:1028000011F40C94071481E0AA81BB818C93009190
:102810008200003081E009F480E08F930091820013
:10282000053E81E009F480E09F9189238F93AA817E
:10283000BB810C91013081E009F080E09F918923F8
:10284000882311F40C94431500918D00003211F08F
:102850000C942E14A5EBB0E00E94CC250027ABE62B
:10286000B0E08C9183FB0EF401E040E0041711F01E
:102870000C94631481E0AC81BD818C93AC85BD85E3
:102880004D915C91A5EBB0E00D911C9104171507DB
:1028900081E009F080E08F93A5EBB0E00D911C91F1
:1028A000003050E0150780E010F009F081E09F91C2
:1028B0008923882311F40C94611480E0AC81BD81DC
:1028C0008C930C94971480E0AC81BD818C9381E053
:1028D000A881B9818C93A881B9810C91053018F039
:1028E00011F00C949714A881B981AD90BB24ACE988
:1028F000B0E0AA0DBB1D4C91A881B981AD90BB245D
:10290000A1E8B0E0AA0DBB1D0C91041711F40C94C2
:102910008F1481E0AC81BD818C930C949714A881B5
:10292000B9818C918F5F8C9311F00C946B14AC81F6
:10293000BD810C91003081E009F080E08F93AC857F
:10294000BD850D911C910F315EE4150781E009F002
:1029500080E09F91892B882311F40C9443150E94E9
:102960007015A885B9850D911D912D913C9140E080
:1029700052E060E070E00E946F26AFE8B0E04D9357
:102980005D936D937D93E3E9F0E0FA93EA935A92B5
:102990004A92AE85BF850D911D912D913C91A42D3C
:1029A000B52D0D931D932D933C9384E00E94B92582
:1029B0000E944917249684E00E94B52580918D00DD
:1029C00080938E00AC85BD850D911C910F315EE426
:1029D000150711F00C941415A8E6B7E0E5EBF0E04C
:1029E0000E948E270E944926EEE7F1E50E945126BB
:1029F000A5EAB0E00E944B26EEE7F1E50E945126E1
:102A000000918D00003111F00C940A15E0E8F1E519
:102A10000E945126A8E6B7E0E885F9850E94912733
:102A20000E9449260E945D26AC81BD810C91003038
:102A300011F00C94431570916B00706170936B00F2
:102A400000918E00003181E009F080E08F93AC8529
:102A5000BD850D911C910F315EE4150781E009F4ED
:102A600080E09F918923882311F40C944315AA8553
:102A7000BB850D911D912D913C91ABECB0E00D9378
:102A80001D932D933C9300918200003011F00C9423
:102A90004E1570916B00706170936B00AE81BF81B9
:102AA0008C918F5F8C9311F00C9489138FEF0E949F
:102AB000FD260E94FF260E94FE26A0E6B0E08C9331
:102AC0008FEF0E94FD260E94FF260E94FE26A0E6B0
:102AD000B0E08C938CE0481A8827580A2C96089509
:102AE00081E00E941927A5EAB0E088278C9381E055
:102AF000A881B9818C93A881B9810C91083018F014
:102B000011F00C94AA15A881B981AD90BB24A1E85D
:102B1000B0E0AA0DBB1D0C91003211F40C94A2156B
:102B2000A881B981AD90BB24A1E8B0E0AA0DBB1D7E
:102B30008C91A5EAB0E08F930E9436268F918D93F9
:102B400088278C93A881B9818C918F5F8C9311F029
:102B50000C947B15A5EAB0E00E943626E4E8F1E586
:102B60000E94302689E0A881B9818C93A881B9811F
:102B70000C910B3018F011F00C94D815A881B98184
:102B8000AD90BB24A1E8B0E0AA0DBB1D8C91A5EAD5
:102B9000B0E08F930E9436268F918D9388278C9377
:102BA000A881B9818C918F5F8C9311F00C94B6152C
:102BB00081E0481A8827580A2296089581E00E94E9
:102BC000192781E00E94192784E00E9419278FEFBE
:102BD0000E94FD260E94FF260E94FE26AC81BD8138
:102BE0008C938FEF0E94FD260E94FF260E94FE26F6
:102BF000AA81BB818C93AA81BB810C9111272227CA
:102C0000332740E051E060E070E00E946A26A8852A
:102C1000B9850D931D932D933D93A885B9850D918D
:102C20001D912D913C91AC81BD814C91552766271A
:102C300077270E947127A885B9850D931D932D9341
:102C40003D93A885B9850D911D912D913C9140E052
:102C500050E061E070E00E946A26A881B9810D937E
:102C60001D932D933D938FEF0E94FD260E94FF261A
:102C70000E94FE26AC81BD818C938FEF0E94FD26C1
:102C80000E94FF260E94FE26AC81BD818C938FEFAF
:102C90000E94FD260E94FF260E94FE26AC81BD8177
:102CA0008C938FEF0E94FD260E94FF260E94FE2635
:102CB000AC81BD818C938FEF0E94FD260E94FF2680
:102CC0000E94FE26AC81BD818C938FEF0E94FD2671
:102CD0000E94FF260E94FE26AA81BB818C93AA81B6
:102CE000BB810C9111272227332740E051E060E09F
:102CF00070E00E946A26A885B9850D931D932D93D7
:102D00003D93A885B9850D911D912D913C91AC8184
:102D1000BD814C915527662777270E947127A8858A
:102D2000B9850D931D932D933D93A885B9850D917C
:102D30001D912D913C91A881B9814D915D916D912D
:102D40007C910E947127A885B9850D931D932D93C1
:102D50003D938FEF0E94FD260E94FF260E94FE26D3
:102D6000AC81BD818C938FEF0E94FD260E94FF26CF
:102D70000E94FE26AA81BB818C93AA81BB810C9103
:102D800011272227332740E051E060E070E00E94E5
:102D90006A26A881B9810D931D932D933D93A88137
:102DA000B9810D911D912D913C91AC81BD814C91CA
:102DB0005527662777270E947127A881B9810D932F
:102DC0001D932D933D938FEF0E94FD260E94FF26B9
:102DD0000E94FE26AC81BD818C938FEF0E94FD2660
:102DE0000E94FF260E94FE26AA81BB818C93AA81A5
:102DF000BB810C9111272227332740E051E060E08E
:102E000070E00E946A26AE81BF810D931D932D93C1
:102E10003D93AE81BF810D911D912D913C91AC816F
:102E2000BD814C915527662777270E947127AE8177
:102E3000BF810D931D932D933D93AE81BF810D9165
:102E40001D912D913C9140E050E061E070E00E94C6
:102E50006A26AE81BF810D931D932D933D93AE8164
:102E6000BF810D911D912D913C91A881B9814D910A
:102E70005D916D917C910E947127AE81BF810D9310
:102E80001D932D933D9386E0481A8827580A26966D
:102E9000089584E00E94192784E00E941927AC81DC
:102EA000BD810D911D912D913C9142E050E060E07B
:102EB00070E00E947627A881B9810D931D932D9310
:102EC0003D93A0E7B0E00C91112722273327A8817A
:102ED000B9814D915D916D917C910E946A26AA8184
:102EE000BB810D931D932D933D93AA81BB810D91C1
:102EF0001D912D913C91A7E7B0E04D915D916D91B1
:102F00007C910E947127AA81BB810D931D932D9303
:102F10003D9300917F000B3011F40C94A117AA810E
:102F2000BB810D911D912D913C9140E250E060E0FC
:102F300070E00E947127AA81BB810D931D932D9390
:102F40003D93AA81BB810D911D912D913C91AE8144
:102F5000BF810D931D932D933C9388E0481A8827D9
:102F6000580A2496089584E00E94192782E00E945E
:102F7000192700917F000B3011F00C94F717AC81EA
:102F8000BD810D911D912D913C9140E850E060E094
:102F900070E00E946F26A2EDB0E04D935D936D93BB
:102FA0007D93AC81BD810D911C9140E850E00E9461
:102FB0000A26A881B9810D931C93A881B9810D912E
:102FC0001C9144E050E00E942426A881B9810D9311
:102FD0001C93A881B9810D911C9144E050E0040F2D
:102FE000151FA881B9810D931C930C942D18AC81E9
:102FF000BD810D911D912D913C9140E051E060E02B
:1030000070E00E946F26A2EDB0E04D935D936D934A
:103010007D93AC81BD810D911C9140E051E00E94F7
:103020000A26A881B9810D931C93A881B9810D91BD
:103030001C9142E050E00E942426A881B9810D93A2
:103040001C93A881B9810D911C9142E050E0040FBE
:10305000151FA881B9810D931C93A2EDB0E00D91CD
:103060001D912D913C91ABE7B0E04D915D916D913B
:103070007C910E947127A2EDB0E00D931D932D93DA
:103080003D93A2EDB0E00D911D912D913C91AEE6E6
:10309000B0E04D915C91662777270E947127A2EDE1
:1030A000B0E00D931D932D933D930E947D1EA8814A
:1030B000B981AD90BC90AFEDB0E0AA0DBB1D8C9175
:1030C000AA81BB818D9388278D938D938C93A88142
:1030D000B9810E94D225AA81BB810D911D912D91AC
:1030E0003C9140E051E060E070E00E946A26AA81D5
:1030F000BB810D931D932D933D93AA81BB810D91AF
:103100001D912D913C91A881B981AD90BC90AFEDFE
:10311000B0E0AA0DBB1D4C915527662777270E946A
:103120007127AA81BB810D931D932D933D9300912F
:103130007F000B3011F00C94FD18A881B9810E941A
:10314000D225AA81BB810D911D912D913C9140E02A
:1031500051E060E070E00E946A26AA81BB810D9375
:103160001D932D933D93AA81BB810D911D912D91AE
:103170003C91A881B981AD90BC90AFEDB0E0AA0DB3
:10318000BB1D4C915527662777270E947127AA817E
:10319000BB810D931D932D933D93A881B9810E940E
:1031A000D225AA81BB810D911D912D913C9140E0CA
:1031B00051E060E070E00E946A26AA81BB810D9315
:1031C0001D932D933D93AA81BB810D911D912D914E
:1031D0003C91A881B981AD90BC90AFEDB0E0AA0D53
:1031E000BB1D4C915527662777270E947127AA811E
:1031F000BB810D931D932D933D93AA81BB810D91AE
:103200001D912D913C91AE81BF810D931D932D9306
:103210003C9386E0481A8827580A2496089581E04E
:103220000E94192781E00E94192709B340EF042367
:10323000AA81BB810C93AA81BB810C9148E00E94BA
:103240004E280C930027BB27A3E38C9184FB0EF43C
:1032500001E041E0041711F00C943319AA81BB81FD
:103260008C918F5F8C93AA81BB818C9180958C937C
:10327000AA81BB810C914FE10423AC81BD810C93E9
:103280000027ABE6B0E08C9185FB0EF401E041E055
:10329000041711F00C945419AA81BB810C914FE0D2
:1032A0000423AC81BD810C9382E0481A8827580A18
:1032B0002496089581E00E941927DF9AAF9ADE9A3A
:1032C000AE9ADD9AAD9ADC9AAC9A80E0AA81BB8175
:1032D0008C93AD98E881F981FA93EA930E94F519ED
:1032E0002296AD9AA881B9810C91003018F011F0A6
:1032F0000C947C190C948619A881B9810C9144E036
:10330000049FAA81BB810C920C94EF19DD98E8818F
:10331000F981FA93EA930E94F5192296DD9AA88121
:10332000B9810C91003018F011F00C9499190C949B
:10333000A919A881B9810C9144E0049F0C92A8813D
:10334000B9810C9141E0041BAA81BB810C930C94C0
:10335000EF19AC98E881F981FA93EA930E94F51984
:103360002296AC9AA881B9810C91003018F011F026
:103370000C94BC190C94CC19A881B9810C9144E02F
:10338000049F0C92A881B9810C9142E0041BAA8190
:10339000BB810C930C94EF19DC98E881F981FA93C6
:1033A000EA930E94F5192296DC9AA881B9810C91C2
:1033B000003018F011F00C94DF190C94EF19A8816B
:1033C000B9810C9144E0049F0C92A881B9810C91C1
:1033D00043E0041BAA81BB810C930C94EF1981E09C
:1033E000481A8827580A2296089581E00E941927D2
:1033F00081E00E941927AA81BB8189B38C93AA819D
:10340000BB818C9180958C93AA81BB810C9140E407
:103410000E944E280C93AA81BB810C91003011F0C0
:103420000C94341AA881B98183B38C93A881B98193
:103430008C9180958C93A881B9810C9140E40E9475
:103440004E280C93A881B9810C91003018F011F02E
:103450000C942C1A0C94341AA881B9810C9142E076
:10346000040FAA81BB810C93AA81BB810C9103300C
:1034700011F00C94411A82E0AA81BB818C930C94C8
:103480004C1AAA81BB810C91023011F00C944C1A99
:1034900083E0AA81BB818C93AA81BB818C91AC8192
:1034A000BD818C9382E0481A8827580A2496089593
:1034B00081E00E94192781E0A881B9818C93AA81BB
:1034C000BB814C91A881B9810C91041718F011F0BF
:1034D0000C94851A5A924A9282E0A42DB52D8C93B1
:1034E00081E00E94B9250E942923229681E00E9452
:1034F000B5258DE790E00E940A27A881B9818C91BB
:103500008F5F8C9311F00C945F1A81E0481A882722
:10351000580A2296089581E00E94192781E0A88127
:10352000B9818C93A881B9810C91063018F011F003
:103530000C94AE1A0E94680D8FE090E00E940A275A
:103540000E946A0D84E690E00E940A27A881B98152
:103550008C918F5F8C9311F00C94921A81E0481A31
:103560008827580A229608950E94F626C39A80E971
:1035700091E00E940A2781B5886081BD0E94EB21FD
:103580005A924A9281E0A42DB52D8C9381E00E943D
:10359000B9250E943722229681E00E94B52581B587
:1035A000886181BD877F81BD88EC90E00E940A27F9
:1035B000FF27E0E1FA93EA935A924A928BE0A42D16
:1035C000B52D8C9381E00E94B9250E94BF242496DA
:1035D00081E00E94B525013051E0150711F00C94EF
:1035E0000A1B5A924A92ADEBB0E08D919C91A42DAA
:1035F000B52D8D939C9382E00E94B9250E94CF2225
:10360000229682E00E94B525E6E8F1E50E94512667
:103610000E945D265A924A9282E3A42DB52D8C9386
:1036200081E00E94B9250E943722229681E00E9403
:10363000B525C29AD89A82E390E00E940A2708959D
:1036400081E00E94192781E00E9419278FEFAA814B
:10365000BB818C9380E0A881B9818C93A881B981CA
:103660000C91073018F011F00C94431B91E0AA81E3
:10367000BB810E94EC26A881B9818C918F5F8C93CD
:1036800011F00C942E1B82E0481A8827580A2496C1
:10369000089581E00E94192781E00E94192781E0A6
:1036A0000E94192782E00E94192782E00E941927B0
:1036B0008FEFAA85BB858C9381E0A885B9858C9313
:1036C000A885B9850C91003418F011F00C94721B88
:1036D0000E94201BA885B9858C918F5F8C9311F077
:1036E0000C94601BC49881E0A885B9858C93A8854B
:1036F000B9850C91003418F011F00C94891B0E94CC
:10370000201BA885B9858C918F5F8C9311F00C9448
:10371000771B8AE090E00E940A27A895EE81FF813E
:10372000FA93EA935A924A9280E4A42DB52D8C9391
:1037300081E00E94B9255A924A9200E010E020E010
:1037400030E0A42DB52D0D931D932D933C9384E073
:103750000E94B9250E945A21269685E00E94B5252F
:10376000AE81BF810C91013011F40C94C01BC49A3E
:10377000EAE8F1E50E9451260E945D260C94771E2E
:1037800081E0AA85BB858C93A89580E090E0A88114
:10379000B9818D939C93EE81FF81FA93EA935A92BB
:1037A0004A9281E4A42DB52D8C9381E00E94B92525
:1037B0005A924A9200E010E020E030E0A42DB52DAE
:1037C0000D931D932D933C9384E00E94B9250E9494
:1037D0005A21269685E00E94B525A881B9810E94CC
:1037E000CC25AE81BF810C91003081E009F080E0F2
:1037F0008F93A881B9810D911C91003050E015077D
:1038000081E009F080E09F91892B882311F40C94CA
:10381000CB1BC49AA881B9810D911C91003050E056
:10382000150711F00C941C1CE2E9F1E50E945126E9
:103830000E945D260C94771EA89584E690E00E9475
:103840000A27A895C49881E090E00E940A27EE819B
:10385000FF81FA93EA935A924A9280E5A42DB52DFE
:103860008C9381E00E94B9255A924A9201E010E0BF
:1038700020E030E0A42DB52D0D931D932D933C93A6
:1038800084E00E94B9250E945A21269685E00E9474
:10389000B52585E090E00E940A27C49A8AE090E06E
:1038A0000E940A27A89500E010E020E030E0ABE796
:1038B000B0E00D931D932D933C9300E010E020E0C9
:1038C00030E0A2EDB0E00D931D932D933C930E9448
:1038D0007D1E00E010E020E030E0A2EDB0E00D93AE
:1038E0001D932D933C930027A0EDB0E08C9184FBB9
:1038F0000EF401E041E0041711F00C94811C0C94CB
:10390000771EA8950091EC00023011F40C94151D5F
:103910008091A20280937F00A9EAB2E00D91112765
:1039200040E051E00E942426AA81BB810D931C93A4
:10393000AA81BB810D911C91A8EAB2E04D91552757
:10394000040F151FAA81BB810D931C93AA81BB8113
:103950000D911C912227332740E050E061E070E098
:103960000E946A26ABE7B0E00D931D932D933D9323
:10397000A7EAB2E00D91112740E051E00E94242611
:10398000AA81BB810D931C93AA81BB810D911C91CF
:10399000A6EAB2E04D915527040F151FAA81BB81FD
:1039A0000D931C93ABE7B0E00D911D912D913C91CF
:1039B000AA81BB814D915C91662777270E94712770
:1039C000ABE7B0E00D931D932D933D9300917F00E5
:1039D0000C3011F00C94EF1C8BE080937F00009171
:1039E0007F000E3011F00C94F81C8BE080937F0068
:1039F00000917F000F3011F00C94011D8BE080933B
:103A00007F00ABE7B0E00D911D912D913C91A2EDAF
:103A1000B0E00D931D932D933C930E947D1EA2ED6B
:103A2000B0E00E94D8250C94691D0091160106345F
:103A300011F00C943F1D84E080937F0087E3A885FC
:103A4000B9858C93A885B9850C910C3318F011F0C9
:103A50000C943D1DA885B985AD90BB24AFEDB0E0B9
:103A6000AA0DBB1D8C910E946026A885B9858C91FA
:103A70008F5F8C9311F00C94221D0E945D260091A3
:103A80003201063411F00C94691D8BE080937F00A5
:103A900083E5A885B9858C93A885B9850C910735F0
:103AA00018F011F00C94671DA885B985AD90BB2462
:103AB000AFEDB0E0AA0DBB1D8C910E946026A885D9
:103AC000B9858C918F5F8C9311F00C944C1D0E94E2
:103AD0005D26ECE9F1E50E945126A8E6B7E0EFE7A4
:103AE000F0E00E949D270E9449260E945D26EEEA92
:103AF000F1E50E945126A8E6B7E0EBE7F0E00E946E
:103B000091270E9449260E945D2684E0A885B985F8
:103B10008C93A885B9850C910B3018F011F00C949A
:103B2000A41DA885B985AD90BB24AFEDB0E0AA0D6A
:103B3000BB1D8C910E946026A885B9858C918F5FF2
:103B40008C9311F00C94891D0E945D268091ED00EC
:103B500080937000E0ECF1E50E945126A8E6B7E002
:103B6000E0E7F0E00E949D270E9449260E945D2622
:103B700000917000003011F00C94C01D0C94771E61
:103B800000917000003418F011F00C94C91D0C94D1
:103B9000CB1D0C94771E8091EE00AE81BF818C937B
:103BA0008091EF00AC81BD818C93AC81BD819C91F3
:103BB000AE81BF818C91AEE6B0E08D939C938091F5
:103BC000F600AE81BF818C938091F700AC81BD81FE
:103BD0008C93AC81BD819C91AE81BF818C91A1E71A
:103BE000B0E08D939C93A1E7B0E00D911C91003063
:103BF00050E0150711F00C94131E80910401AE8162
:103C0000BF818C9380910501AC81BD818C93AC8187
:103C1000BD819C91AE81BF818C91A1E7B0E08D9375
:103C20009C930C94131EA1E7B0E00D911C91003001
:103C300050E0150711F00C941F1E0C94771E02E043
:103C400010E020E030E0A1E7B0E04D915C91662704
:103C500077270E946A26A3E7B0E00D931D932D936A
:103C60003D93A3E7B0E00D911D912D913C91AEE6FF
:103C7000B0E04D915C91662777270E947127A3E7FA
:103C8000B0E00D931D932D933D93A3E7B0E00D910C
:103C90001D912D913C91A2EDB0E04D915D916D9102
:103CA0007C910E947127A3E7B0E00D931D932D93A3
:103CB0003D93E0EDF1E50E945126A8E6B7E0E3E789
:103CC000F0E00E9491270E9449260E945D26A3E70A
:103CD000B0E00D911D912D913C91A2EDB0E00D93BE
:103CE0001D932D933C9380E0AA85BB858C9387E040
:103CF000481A8827580A2A96089581E00E941927B1
:103D000081E00E94192782E00E94192782E00E9428
:103D100019278FEFAE81BF818C9391E0AE81BF8177
:103D20000E94EC2691E0AE81BF810E94EC2691E0DA
:103D3000AE81BF810E94EC2691E0AE81BF810E94DE
:103D4000EC2691E0AE81BF810E94EC2691E0AE812D
:103D5000BF810E94EC2691E0AE81BF810E94EC26DB
:103D600091E0AE81BF810E94EC2691E0AE81BF81DF
:103D70000E94EC2691E0AE81BF810E94EC2691E08A
:103D8000AE81BF810E94EC2691E0AE81BF810E948E
:103D9000EC2691E0AE81BF810E94EC2691E0AE81DD
:103DA000BF810E94EC2691E0AE81BF810E94EC268B
:103DB00091E0AE81BF810E94EC26C49880E090E043
:103DC000A881B9818D939C938FEF0E94FD260E945C
:103DD000FF260E94FE26AE81BF818C93A881B98107
:103DE0000E94CC25AE81BF810C91003081E009F4A6
:103DF00080E08F93A881B9810D911C91003050E033
:103E0000150781E009F080E09F91892B882311F448
:103E10000C94E41EA881B9810D911C91003050E0F2
:103E2000150711F00C94211FE8EDF1E50E945126D1
:103E30000E945D267091D00070617093D0000C9448
:103E40006E20EE81FF81FA93EA935A924A9281E5BD
:103E5000A42DB52D8C9381E00E94B9255A924A92E7
:103E6000A2EDB0E00D911D912D913C91A42DB52DA9
:103E70000D931D932D933C9384E00E94B9250E94DD
:103E80005A21269685E00E94B5250027A0EDB0E0D6
:103E90008C9184FB0EF401E041E0041711F00C94C6
:103EA000611FE6EEF1E50E945126A8E6B7E0E2EDDB
:103EB000F0E00E9491270E9449260E945D260C9402
:103EC0006E20A895AE81BF810C91003011F00C944A
:103ED000AC1F80E090E0A881B9818D939C938FEF17
:103EE0000E94FD260E94FF260E94FE26AE81BF8111
:103EF0008C93A881B9810E94CC25AE81BF810C91A1
:103F0000003081E009F480E08F93A881B9810D91A0
:103F10001C91003050E0150781E009F080E09F918E
:103F2000892B882311F40C946F1FA881B9810D91FE
:103F30001C91003050E0150711F00C94AC1FE0E02C
:103F4000F2E50E9451260E945D267091D0007061BA
:103F50007093D0000C946E20AE81BF810C910F3F06
:103F600011F00C94F61F80E090E0A881B9818D9348
:103F70009C938FEF0E94FD260E94FF260E94FE2642
:103F8000AE81BF818C93A881B9810E94CC25AE817E
:103F9000BF810C910F3F81E009F480E08F93A881ED
:103FA000B9810D911C91003050E0150781E009F0B6
:103FB00080E09F91892B882311F40C94B91FA8816C
:103FC000B9810D911C91003050E0150711F00C944F
:103FD000F61FEEE0F2E50E9451260E945D267091E8
:103FE000D00070617093D0000C946E20AE81BF81C0
:103FF0000C910E3F11F40C941320ECE1F2E50E94B9
:104000005126A8E6B7E0EE81FF810E949D270E941D
:1040100049260E945D26C49A7091D0007061709309
:10402000D0000C946E2080E090E0AA81BB818D933B
:104030009C9380E0AE81BF818C93AE81BF810C9157
:104040000F3F18F011F00C945520AA81BB810E94FB
:10405000CC258FEF0E94FD260E94FF260E94FE269F
:10406000AA81BB81AD90BC90AFEDB0E0AA0DBB1DA5
:104070008C93AA81BB810E94CC258FEF0E94FD26E4
:104080000E94FF260E94FE26AA81BB81AD90BC90B3
:10409000AFEDB0E0AA0DBB1D8C93AE81BF818C91BA
:1040A0008F5F8C9311F00C941D208FEF0E94FD26E2
:1040B0000E94FF260E94FE26AE81BF818C938FEF67
:1040C0000E94FD260E94FF260E94FE26AE81BF812F
:1040D0008C93C49AA2EDB0E00E94BD2586E0481AF8
:1040E0008827580A2896089582E00E94192781E0BF
:1040F0000E94192780E0AE81BF818C930E94201B13
:10410000C49880E090E0AA81BB818D939C938FEF4F
:104110000E94FD260E94FF260E94FE26A881B981EA
:104120008C93AA81BB810E94CC25A881B9810C9176
:10413000003081E009F480E08F93AA81BB810D916A
:104140001C91003050E0150781E009F080E09F915C
:10415000892B882311F40C948720AA81BB810D91AF
:104160001C91003050E0150711F00C94C420E8EDCC
:10417000F1E50E9451260E945D267091D000706189
:104180007093D0000C945421E881F981FA93EA935A
:104190005A924A9281E5A42DB52D8C9381E00E941C
:1041A000B9255A924A92AA85BB850D911D912D91F0
:1041B0003C91A42DB52D0D931D932D933C9384E03C
:1041C0000E94B9250E945A21269685E00E94B525B5
:1041D000A881B9810C91003011F00C941B2180E072
:1041E00090E0AA81BB818D939C938FEF0E94FD2666
:1041F0000E94FF260E94FE26A881B9818C93AA8185
:10420000BB810E94CC25A881B9810C91003081E04E
:1042100009F480E08F93AA81BB810D911C9100303D
:1042200050E0150781E009F080E09F91892B8823F9
:1042300011F40C94F520A881B9810C910F3F11F075
:104240000C944E2180E090E0AA81BB818D939C93D9
:104250008FEF0E94FD260E94FF260E94FE26A88165
:10426000B9818C93AA81BB810E94CC25A881B98198
:104270000C910F3F81E009F480E08F93AA81BB810C
:104280000D911C91003050E0150781E009F080E0AD
:104290009F91892B882311F40C942821A881B9813E
:1042A0008C91AE81BF818C9383E0481A8827580A8D
:1042B0002496089584E00E94192781E00E9419271E
:1042C00082E00E9419278FEFAA81BB818C9391E035
:1042D000AA81BB810E94EC2691E0A885B9850E9445
:1042E000EC26AE81BF810D911D912D913C9140E056
:1042F00052E060E070E00E946A26AC81BD810D93BF
:104300001D932D933D93AC81BD818F9314968E9117
:104310000E94E0218E910E94E0218E910E94E02176
:104320008E910E94E02185E90E94E0218F9180E03A
:1043300090E0A881B9818D939C938FEF0E94FD2618
:104340000E94FF260E94FE26AA81BB818C93A88131
:10435000B9810E94CC25AA81BB810C910F3F81E0DD
:1043600009F480E08F93A881B9810D911C910030F0
:1043700050E0150781E009F080E09F91892B8823A8
:1043800011F40C949D21A881B9810D911C910030EC
:1043900050E0150711F00C94D821EAE2F2E50E94F2
:1043A00051260E945D267091D00070617093D000FC
:1043B000AA81BB818C91AA85BB858C930C94E52145
:1043C0008FB9779BFECF8FB1089587E0481A882771
:1043D000580A269608955A924A9284E298E0A42DAB
:1043E000B52D8D939C9382E00E94B9255A924A92F2
:1043F00080E0A42DB52D8C9381E00E94B9250E9408
:104400006424249683E00E94B525EF93FF93ECE8A3
:10441000F1E00E94DE26FF91EF91BB27A0E38C9193
:1044200082FBDEF789E190E00E940A275A924A92C5
:1044300080E298E0A42DB52D8D939C9382E00E949C
:10444000B9255A924A9280E0A42DB52D8C9381E033
:104450000E94B9250E946424249683E00E94B52519
:1044600089E190E00E940A270E94EC22089582E0F0
:104470000E94192700E011E0AA81BB814D915527C8
:104480000E942426A881B9810D931C93A881B9812B
:104490000D911C91AA81BB814D915527040F151FC9
:1044A000A881B9810D931C935A924A92AA81BB812B
:1044B0008D919C91A42DB52D8D939C9382E00E94AB
:1044C000B9255A924A928BE0A42DB52D8C9381E0A8
:1044D0000E94B9250E946424249683E00E94B52599
:1044E0005A924A9280E298E0A42DB52D8D939C9328
:1044F00082E00E94B9255A924A9280E0A42DB52DFF
:104500008C9381E00E94B9250E946424249683E064
:104510000E94B52582E0481A8827580A22960895F5
:1045200082E00E94192700E110E0AC81BD814D912D
:1045300055270E942426A881B9810D931C93A88138
:10454000B9810D911C91AA81BB814D915527040F12
:10455000151FA881B9810D931C935A924A92AA8182
:10456000BB818D919C91A42DB52D8D939C9382E060
:104570000E94B9255A924A9282E0A42DB52D8C93BF
:1045800081E00E94B9250E946424249683E00E9461
:10459000B52582E0481A8827580A229608955A922B
:1045A0004A92AA81BB818D919C91A42DB52D8D93AA
:1045B0009C9382E00E94B9255A924A9283E0A42DEE
:1045C000B52D8C9381E00E94B9250E946424249625
:1045D00083E00E94B525089581E00E94192781E0BB
:1045E0000E941927C49AD898C29880E0A881B981FE
:1045F0008C9380E0AA81BB818C93AA81BB810C91B2
:104600000F3118F011F00C94212391E0A881B981A9
:104610000E94EC2691E0A881B9810E94EC2691E0ED
:10462000A881B9810E94EC2691E0A881B9810E94FD
:10463000EC26AA81BB818C918F5F8C9311F00C9436
:10464000FD22C29AD89A82E0481A8827580A2496EE
:10465000089581E00E9419275A924A9280E298E0D8
:10466000A42DB52D8D939C9382E00E94B9255A927A
:104670004A9280E0A42DB52D8C9381E00E94B9254B
:104680000E946424249683E00E94B525AA81BB8100
:104690000C91003011F00C945C235A924A9280E005
:1046A000A42DB52D8C9381E00E94B9250E94D623BC
:1046B000229681E00E94B525AA81BB810C91013030
:1046C00011F00C9472235A924A9285E6A42DB52DCE
:1046D0008C9381E00E94B9250E94D623229681E026
:1046E0000E94B525AA81BB810C91023011F00C9477
:1046F0009F235A924A9283E6A42DB52D8C9381E094
:104700000E94B9250E94D623229681E00E94B525F9
:1047100088EC90E00E940A275A924A9280E0A42DE9
:10472000B52D8C9381E00E94B9250E94D623229654
:1047300081E00E94B52582E390E00E940A27AA81C9
:10474000BB810C91033011F00C94C8235A924A9209
:1047500082E6A42DB52D8C9381E00E94B9250E949C
:10476000D623229681E00E94B52580E991E00E943F
:104770000A275A924A9280E0A42DB52D8C9381E0AD
:104780000E94B9250E94D623229681E00E94B52579
:104790008AE090E00E940A278AE090E00E940A27BF
:1047A00081E0481A8827580A2296089581E00E94DD
:1047B0001927C49AD898C298AA81BB810C9100305D
:1047C00018F011F00C94E6230C94202483E5A881C2
:1047D000B9818C9391E0A881B9810E94EC268FEE7B
:1047E000A881B9818C9391E0A881B9810E94EC26BF
:1047F0008EE6A881B9818C9391E0A881B9810E944D
:10480000EC2691E0AA81BB810E94EC2680E0A88181
:10481000B9818C9391E0A881B9810E94EC2691E046
:10482000A881B9810E94EC2691E0A881B9810E94FB
:10483000EC2691E0A881B9810E94EC260C945C24BE
:1048400085E4A881B9818C9391E0A881B9810E9407
:10485000EC2688E7A881B9818C9391E0A881B98181
:104860000E94EC2689E6A881B9818C9391E0A88109
:10487000B9810E94EC2684E7A881B9818C9391E0EC
:10488000A881B9810E94EC2680E0A881B9818C932F
:1048900091E0A881B9810E94EC2691E0A881B981BC
:1048A0000E94EC2691E0A881B9810E94EC2691E05B
:1048B000A881B9810E94EC26C29AD89A81E0481A50
:1048C0008827580A2296089581E00E941927C29AE3
:1048D000D8985A924A9282E0A42DB52D8C9381E00B
:1048E0000E94B9250E941925229681E00E94B525D3
:1048F0005A924A92AC81BD818C91A42DB52D8C9396
:1049000081E00E94B9250E941925229681E00E942B
:10491000B525AC81BD8111968C91A881B9818C930C
:104920005A924A92AA81BB818C91A42DB52D8C9369
:1049300081E00E94B9250E941925229681E00E94FB
:10494000B525AC81BD818C91A881B9818C935A9297
:104950004A92AA81BB818C91A42DB52D8C9381E0C4
:104960000E94B9250E941925229681E00E94B52552
:10497000D89A81E0481A8827580A2296089581E03B
:104980000E94192781E00E94192782E00E941927BE
:10499000C29AD8985A924A9283E0A42DB52D8C934E
:1049A00081E00E94B9250E941925229681E00E948B
:1049B000B5255A924A92A885B9858C91A42DB52D1A
:1049C0008C9381E00E94B9250E941925229681E0EE
:1049D0000E94B525EC81FD81FA93EA930E941F2580
:1049E0002296EA81FB81FA93EA930E941F25229680
:1049F000D89AAC81BD810D91112740E051E00E9411
:104A00002426A881B9810D931C93A881B9810D91A9
:104A10001C91AA81BB814D915527040F151FA885B4
:104A2000B9850D931C9384E0481A8827580A269666
:104A3000089591E0A881B9810E94EC26089581E053
:104A40000E94192791E0A881B9810E94E126A881DE
:104A5000B9818C91AA81BB818C9381E0481A882707
:104A6000580A2296089582E00E94192781E00E9448
:104A70001927C49ABB27A0E38C9182FBDEF7C2986A
:104A8000AC81BD810D911C91003052E0150711F0F1
:104A90000C94822581E090E0AA81BB818D939C9348
:104AA00080E0A881B9818C93A881B9810C910F30E5
:104AB00018F011F00C948025BB27A0E38C9182FBA9
:104AC000DEF790E2AA81BB81AD90BC90AFEDB0E083
:104AD000AA0DBB1D0E94EC26AA81BB810D911C91E1
:104AE00040E250E0040F151FAA81BB810D931C9377
:104AF000A881B9818C918F5F8C9311F00C9454250F
:104B00000C94AE2581E090E0AA81BB818D939C93AB
:104B1000AC81BD814D915C91AA81BB810D911C91AD
:104B20000417150718F011F00C94AE25BB27A0E36D
:104B30008C9182FBDEF7C29A91E0AA81BB81AD9095
:104B4000BC90AFEDB0E0AA0DBB1D0E94EC26AA817F
:104B5000BB810E94CC2511F00C948825C29A83E079
:104B6000481A8827580A24960895481A8827580A08
:104B70000895480E8827581E08950D911D912D9176
:104B80003C9181E0080F8827181F281F381F3C938D
:104B90002E931E930E930895ED91FC913196FC9304
:104BA000EE930895ED91FC913197FC93EE93089567
:104BB0000D911D912D913C910150104020403040AD
:104BC0003C932E931E930E93089508D03DD000FC85
:104BD00010D0089503D01ED001F8F9CF0024E89436
:104BE00057FF02C009D0689400F80BD010F80124D8
:104BF000089502D009D00895509540954F5F5F4FBA
:104C00000895E89417FF0895009510950F5F1F4FC2
:104C100068940895352F242FE894452B11F4689457
:104C20000895512F402F0027112780E1440F551F71
:104C3000001F111F021B130B416018F4020F131FFA
:104C40004E7F8A9599F708950F92049F202C312C5E
:104C5000419F300C509F030C022D102D0F90089592
:104C6000C8950D9231960020D9F708958F938D91B4
:104C70008823E9F711978F91089581E05F9B88273A
:104C8000089588275F9B089500C05F9BFECF8CB17D
:104C90000895A8E6B7E08D91882311F011D0FBCFDD
:104CA00008950E941F27802D11F00AD0FACF089591
:104CB0008D9106D03A95E1F708958DE001D08AE014
:104CC0005D9BFECF8CB9089588EE93E0A3D0319719
:104CD000D9F7089550D00AD000FC05D008954BD0E4
:104CE00020D001F8F9CF52D05AD00895842F952FB3
:104CF000A62FB72F4427552766277727F1E28894F8
:104D000009C020F4480F591F6A1F7B1F76956795CD
:104D1000579547953795279517950795FA9589F7EC
:104D20000895842F952FA62FB72FE894452B462B57
:104D3000472B11F468940895402F512F622F732F41
:104D40000027112722273327F0E2440F551F661F43
:104D5000771F001F111F221F331F081B190B2A0B5F
:104D60003B0B416028F4080F191F2A1F3B1F4E7F81
:104D7000FA9559F708950024E89477FF02C006D009
:104D8000689400F809D010F80124089512D04F5FFC
:104D90005F4F6F4F7F4F0895E89437FF0895009558
:104DA0001095209530950F5F1F4F2F4F3F4F689400
:104DB0000895409550956095709508953197F1F755
:104DC00008950E94FD268C910E94FF268D939A954E
:104DD000D1F70E94FE2608950E94FD268D910E9423
:104DE000FF269A95D9F70E94FE260895BF9ABE988D
:104DF000C69ABD9A80E58DB90895089508958FB932
:104E0000779BFECF8FB10895689462F80895E89477
:104E100062F80895EF93FF93EE27E82BE92B31F02A
:104E2000E0EDF7E03197F1F70197D1F7FF91EF91BE
:104E300008955A924A92480E8827581E0895C89598
:104E4000319600200895819104D08D938823D9F75D
:104E50000895813618F08B3708F48F7D089580E32C
:104E60000EF4839508952E2E3F2E992781918D3231
:104E700009F093958823D1F79A95E22DF32D11230C
:104E800061F0091718F011F0101B01C0191B28F070
:104E900021F080E28D931A95E9F780818D3219F423
:104EA0008D93319604C0222311F08BE28D93091764
:104EB00038F031F0091B21F080E38D930A95E9F772
:104EC00081918D938823E1F7332351F0EA2FFB2F53
:104ED000319633958E9182933A95E1F78EE28C93D9
:104EE0000895040F151F261F371F0895041B150B67
:104EF000260B370B08950417150726073707089563
:104F0000000F111F221F331F089500951095209543
:104F100030950F5F1F4F2F4F3F4F08950191108124
:104F20000EC001911191219130810BC0019110812E
:104F300017FF05C03FEF2FEF04C000811127222784
:104F4000332737FF03C0E1DF8DE28D93CF93DF93EB
:104F5000CF92DF92EF92AA24BB24CC24DD24EE244E
:104F600040E2CAE0DD2755E093E38881890F87FDA1
:104F70009F7083FD907F891B89935A95A9F7C0DFA5
:104F8000AA1CBB1CCC1CDD1CEE1C4A9551F7E894F6
:104F9000EFE0FF2782910ED0EB30E0F71EF068942F
:104FA0008A2D0CD088278D93EF90DF90CF90DF91E2
:104FB000CF910895982F829501D0892F8F70805DB1
:104FC00026F0803309F4089568948D93089500279E
:104FD0001127222733271DD08A3328F4803318F075
:104FE00005D015D0F9CF0EF490CF089580538F934C
:104FF000402F512F622F732F83DF82DF72DF80DF1C
:105000008F919927080F191F291F391F08958D9116
:105010000895E894FCDF8032E9F38B32D9F38930CC
:10502000C9F38D3211F46894F2CF089588278D93D7
:10503000089581918D938823E1F7089509919191C5
:10504000992351F08A95D9F7319781918D930A95DB
:1050500019F08823D1F70895E9CFE199FECFEEBB8F
:10506000FFBB3196089591E001C092E07B3751F487
:105070007FB7F894F2DF8D918DBBE29AE19A9A9511
:10508000C9F77FBF7727089591E001C092E0E5DF7F
:10509000E09A8DB38D939A95D1F70895FF93881B6D
:1050A000F9E0001FFA9511F4FF910895881F841B01
:1050B00018F4840F8894F5CF0894F3CF8FEF83957D
:1050C0009D919923E1F70895689401C0E894AF9306
:1050D000BF938D9116F0919103C00E941F27902DD0
:1050E000891718F011F48823A1F7BF91AF910895A3
:1050F0005069636F4A62205265616C6974792D53FF
:10510000797320342E360000454570726F6D200093
:105110002C004B45593136204F4E00004B4559313C
:1051200036204F4646004D4D4320696E697420007D
:105130007265747279202E2E2E0044535020696EB1
:10514000697420004F0021005A0031003200330002
:10515000340035003600370038003900300059007F
:105160005700520048004E005000420058004400D2
:10517000450056004D005300540049004C002000EB
:10518000442000002E006F6B00004E6F20636172A0
:105190006400426164206361726400005061727453
:1051A0006974696F6E2074797065203A00005061EF
:1051B00072746974696F6E2073746172743A00005E
:1051C000536563742F636C757374657220203A00A5
:1051D000526F6F74203A00005265616420657272EC
:1051E0006F722031000052656164206572726F72C7
:1051F0002032206F6E20736563746F723A20000056
:1052000052656164206572726F72203300005265CE
:105210006164206572726F722034000052656164AF
:10522000206572726F7220350000526561642074CF
:08523000696D656F75740000E3
:00000001FF
